S01800006275696C642F6D6963617A2F6D61696E2E73726563E5
S11300000C945B010C942D150C9437150C9441152C
S11300100C944B150C9455150C945F150C946915A0
S11300200C9499150C9478010C9478010C94341464
S11300300C9467130C941E140C940C150C94E0127D
S11300400C9420130C94A3150C9453170C9478015E
S11300500C94A1170C9478010C9478010C947801F9
S11300600C9429140C9478010C9478010C94780164
S11300700C9478010C9478010C948F170C947801EB
S11300800C948F180C9478010C947801F00B800C6C
S1130090370D3D0D410D740D7A0DA40DB30DFB0DFF
S11300A0070EC40EC80E340F1E1027102E106D102C
S11300B000081C18141000002110422063308440F2
S11300C0A550C660E770088129914AA16BB18CC123
S11300D0ADD1CEE1EFF13112100273325222B5529A
S11300E09442F772D662399318837BB35AA3BDD373
S11300F09CC3FFF3DEE36224433420040114E6646A
S1130100C774A44485546AA54BB528850995EEE5C2
S1130110CFF5ACC58DD55336722611163006D77679
S1130120F6669556B4465BB77AA719973887DFF712
S1130130FEE79DD7BCC7C448E5588668A778400841
S1130140611802282338CCC9EDD98EE9AFF9488962
S113015069990AA92BB9F55AD44AB77A966A711AD9
S1130160500A333A122AFDDBDCCBBFFB9EEB799BB2
S1130170588B3BBB1AABA66C877CE44CC55C222C29
S1130180033C600C411CAEED8FFDECCDCDDD2AAD02
S11301900BBD688D499D977EB66ED55EF44E133EB9
S11301A0322E511E700E9FFFBEEFDDDFFCCF1BBF52
S11301B03AAF599F788F8891A981CAB1EBA10CD12C
S11301C02DC14EF16FE18010A100C230E320045034
S11301D0254046706760B9839893FBA3DAB33DC3A7
S11301E01CD37FE35EF3B1029012F322D232354284
S11301F0145277625672EAB5CBA5A89589856EF537
S11302004FE52CD50DC5E234C324A01481046674D3
S1130210476424540544DBA7FAB79987B8975FE786
S11302207EF71DC73CD7D326F2369106B016576623
S11302307676154634564CD96DC90EF92FE9C8990E
S1130240E9898AB9ABA94458654806782768C01873
S1130250E1088238A3287DCB5CDB3FEB1EFBF98BE6
S1130260D89BBBAB9ABB754A545A376A167AF10AC3
S1130270D01AB32A923A2EFD0FED6CDD4DCDAABDF6
S11302808BADE89DC98D267C076C645C454CA23C13
S1130290832CE01CC10C1FEF3EFF5DCF7CDF9BAFC6
S11302A0BABFD98FF89F176E367E554E745E932E63
S11302B0B23ED10EF01E11241FBECFEFD0E1DEBF3F
S11302C0CDBF11E0A0E0B1E0EEEDF5E300E00BBF3F
S11302D002C007900D92A431B107D9F716E0A4E14A
S11302E0B1E001C01D92AE3EB107E1F70C940011DC
S11302F00C9400008FB7F894992708958FBF089540
S11303008FB7F894282F33278BB391E089278BBBC1
S11303102FBF0895982F8FB7F894282FE92FFF2720
S1130320EA53F94F80818F3FB1F48091DB0689173E
S113033091F08091C3068F3F19F49093C30607C0D0
S11303408091DB06E82FFF27EA53F94F90839093BF
S1130350DB0680E001C085E02FBF99270895282F90
S11303608FB7F89499272CB95E9A8FBF80E090E0FC
S1130370089520E08FB7F894982F8091B7068A30BB
S113038029F48091E305843009F421E09FBF2223FE
S113039051F08FE00E948A018FB7F8949927109248
S11303A025018FBF08958FB7F894282F332781E054
S11303B0809325012FBF0895CF938FB7F894C82F4A
S11303C080919D03882341F48DE00E948A01882353
S11303D019F481E080939D03CFBFCF9108958823C2
S11303E011F06E9A08956E98089580912A018823D9
S11303F019F480E090E0089581E090E008952F9250
S11304003F924F925F926F927F928F929F92AF92A0
S1130410BF92CF92DF92EF92FF920F931F93CF93ED
S1130420DF93CDB7DEB72A970FB6F894DEBF0FBEC1
S1130430CDBF8FB7F894282F332729873A87209088
S11304408E0330908F034090900350909103662464
S11304502EE4A22E93E8B92EC62CD62CE62CF62C2C
S1130460062D162D222D332D442D552D662D762D3A
S1130470862D962D0E949A1829833A834B835C8398
S11304806D837E838F839887822E932EA42EB52E20
S1130490C62ED72EE82EF92E2401350176946794C2
S11304A05794479400E2282D392D4A2D5B2D6C2D4D
S11304B07D2D8E2D9F2D0E94A419A22EB32EC42E05
S11304C0D52EC601B501640D751D861D971D97FFB8
S11304D005C09F776F5F7F4F8F4F9F4F60938E0351
S11304E070938F03809390039093910339853FBF5A
S11304F02A960FB6F894DEBF0FBECDBFDF91CF9121
S11305001F910F91FF90EF90DF90CF90BF90AF902D
S11305109F908F907F906F905F904F903F902F901F
S1130520089580E8809348011092E4051092D40560
S11305301092DD060895CF93DF938FB7F894682F58
S11305407727A091D505B091D605C091D705D09154
S1130550D80582B706B600FE04C01196C11DD11D90
S113056082B7282F33274427552788279A2FAB2F64
S1130570BC2F822B932BA42BB52B6FBFBC01CD01B9
S1130580DF91CF910895FC018285992708958FB753
S1130590F894682F77278091490190914A012CB5EE
S11305A03DB506B602FE03C001962CB53DB5AA279B
S11305B0BB2744275527DC0199278827822B932BB7
S11305C0A42BB52B6FBFBC01CD010895AF92BF9290
S11305D0CF92DF92EF92FF920F931F93CF93DF930B
S11305E00E949B027B018C01C091C605D091C70576
S11305F0E091C805F091C905A0909203B0909303CF
S1130600C0909403D09095039E01AF012A0D3B1D29
S11306104C1D5D1DDA01C9018E199F09A00BB10B98
S1130620EC16FD060E071F0730F02C173D074E078A
S11306305F0778F005C02C173D074E075F0728F4C5
S1130640E216F3060407150720F080E090E0A0E02E
S1130650B0E0813021E0920720E0A20720E0B20759
S113066088F0803030E0930731E0A30730E0B3072F
S113067010F08FEF04C0892F9A2FAB2FBB278093E4
S1130680CB0571C01092CB0581389105A105B10548
S113069048F120E830E040E050E0E20EF31E041F91
S11306A0151FE092C605F092C7050093C805109384
S11306B0C90520E83FEF4FEF5FEFE20EF31E041F82
S11306C0151F820F931FA41FB51F8093920390934D
S11306D09303A0939403B093950380E890E0A0E083
S11306E0B0E014C0CA0DDB1DEC1DFD1DC093C60592
S11306F0D093C705E093C805F093C90510929203FF
S11307001092930310929403109295036E2D982FD8
S113071082B7923008F492E0960F292F2250861760
S113072070F0261740F0821730F082B78E5F00B663
S113073001FCFDCF0DC000B601FCFDCF0EC0261795
S113074010F4821738F082B78E5F00B601FCFDCF3B
S113075081BF04C000B601FCFDCF91BF82E086BF1B
S113076087B7826087BFDF91CF911F910F91FF9070
S1130770EF90DF90CF90BF90AF9008950F931F93A9
S1130780DC01CB016FB7F894062F11278093C605BF
S11307909093C705A093C805B093C905209392030D
S11307A03093930340939403509395030E94E6027D
S11307B00FBF1F910F910895AF92BF92CF92DF9216
S11307C0EF92FF920F931F93CF93DF930E94C70280
S11307D0FC01EB018091960390919703A0919803FB
S11307E0B0919903A090B306B090B406C090B5063A
S11307F0D090B6069C01AD012A0D3B1D4C1D5D1D1C
S113080079018A01EC1AFD0A0E0B1F0BC817D907D0
S1130810EA07FB0730F0281739074A075B0770F02F
S113082005C0281739074A075B0728F4C217D307FE
S1130830E407F50718F0EE24FF24870121E0E2160F
S113084020E8F20620E0020720E0120730F1C05051
S1130850D048EF4FFF4FC0939603D0939703E09394
S11308609803F0939903C050D048E040F04080E0F2
S113087090E8AFEFBFEFE80EF91E0A1F1B1FE092CE
S1130880B306F092B4060093B5061093B606E12CB5
S1130890A0E8FA2E012D112D14C08A0D9B1DAC1D4C
S11308A0BD1D8093960390939703A0939803B093F0
S11308B099031092B3061092B4061092B5061092E2
S11308C0B606BE0197014CB55DB52330310510F471
S11308D023E030E0CB01820F931F9C012350304072
S11308E04617570720F02617370750F003C026177E
S11308F0370718F44217530718F08CB59DB50396C3
S11309009BBD8ABD80E186BF87B7806187BFDF91C9
S1130910CF911F910F91FF90EF90DF90CF90BF90F8
S1130920AF9008950F931F93DC01CB016FB7F89438
S1130930062F11278093960390939703A09398030F
S1130940B09399032093B3063093B4064093B5064D
S11309505093B6060E94DC030FBF1F910F910895B8
S1130960EF92FF920F931F93CF938FB7F894C82FF2
S11309700E94FF01DC01CB019C01277030702F5FC6
S11309803F4FC1F0C901B3E0880F991FBA95E1F751
S1130990820F931F820F931F7C01002711270E944F
S11309A0C702DC01CB01A8019701BC01CD010E9463
S11309B0920406C081E090E090932801809327017F
S11309C0CFBFCF911F910F91FF90EF90089597B7EC
S11309D09F7D97BF90E296BF882319F08EB58064FF
S11309E002C08EB58F7B8EBD87B7806287BF80E0E3
S11309F090E00895FB018FB9779BFECF8FB1808380
S1130A000895EF92FF920F931F93CF93DF93CDB787
S1130A10DEB721970FB6F894DEBF0FBECDBF7B01C2
S1130A208E010F5F1F4FB8010E94FA048F2D992782
S1130A30B8010E94FA04B8018E2D0E94FA0489813B
S1130A40992721960FB6F894DEBF0FBECDBFDF9174
S1130A50CF911F910F91FF90EF900895AF92BF92A5
S1130A60CF92DF92FF920F931F93CF93DF93CDB773
S1130A70DEB721970FB6F894DEBF0FBECDBF5A0183
S1130A80F22E8C01060F111D6E010894C11CD11C9D
S1130A90B601802F80680E94FA0416950795B60166
S1130AA0802F807C0E94FA04FF2041F0B601F501FA
S1130AB081915F010E94FA04FA94F6CF8981992703
S1130AC021960FB6F894DEBF0FBECDBFDF91CF9154
S1130AD01F910F91FF90DF90CF90BF90AF9008953A
S1130AE0882311F06F9A08956F9808951F9310E06A
S1130AF0812F0E94EF01BA9ABB98B99AB89A6C9A5E
S1130B00C098812F0E947005709A6B986A986898B3
S1130B1081E00E94EF011F9108950F931F93CF93DB
S1130B20082F8FB7F894282F3327122F80912C0188
S1130B30882321F02FBF85E090E033C090912A01F3
S1130B40992341F482E080932A0190930C0180E080
S1130B5090E003C080910C019927882351F08230E2
S1130B6059F410920B0120910C01109229012223B7
S1130B7019F480E090E002C085E090E09927C82F46
S1130B80882311F40E9476058C2F9927282F882317
S1130B9029F400930D0181E080932C011FBF822F63
S1130BA09927CF911F910F910895CF93C82F0E9439
S1130BB0F501882311F40E94760580912A01882387
S1130BC059F481E080932A01C0930B018AE00E94CA
S1130BD08A0180E090E025C080910C01823019F4F4
S1130BE08BE00E948A01EC2FFF27E55BFE4F80819A
S1130BF08F3FA1F4E0910901EC1781F080910A0183
S1130C008F3F19F4C0930A0104C0FF27E55BFE4F30
S1130C10C083C093090180E090E002C085E090E0C9
S1130C2099279927CF910895CF93282F8FB7F894B8
S1130C30C82F90912C01992369F081E090E002C0C3
S1130C40880F991F2A95E2F720912B01282B2093D6
S1130C502B0108C020930D0181E080932C01892F82
S1130C600E94D505CFBF80E090E0CF910895CF9347
S1130C7082E00E948D059927C82F882319F082E00D
S1130C800E9414068C2F9927CF9108951F93CF9318
S1130C90DF93982F8FB7F894282F3327122F809142
S1130CA00D01891711F02FBF6AC02FEF20930D019A
S1130CB080912A018230D9F580910C018823B9F5FD
S1130CC080912901882329F080910B0180930C01E4
S1130CD02EC020930C0190910A019F3F31F1E92F1E
S1130CE0FF27E55BFE4F808180930A018F3F11F45B
S1130CF020930901208390930B0181E080932A01C2
S1130D008AE00E948A0113C020930D0181E090E0E3
S1130D1002C0880F991F4A95E2F7809538233093D3
S1130D202B0180E00E94D50529C080932A010E94EE
S1130D30F501C82FDD27CC2331F48C2F0E94EF015D
S1130D40C093DC06C09A30912B013323A9F0209183
S1130D500D012F5F632F7727243008F020E0422F06
S1130D605527CB01042E02C0959587950A94E2F786
S1130D7080FDCACF2F5FF0CF10922C011FBFDF91EF
S1130D80CF911F9108951F93CF93DF93CDB7DEB713
S1130D9023970FB6F894DEBF0FBECDBF11E0C09805
S1130DA08091CA05882341F0BE016F5F7F4F85E0C3
S1130DB00E94FA04898107C0BE016E5F7F4F84E000
S1130DC00E94FA048A8183FD09C0BE016D5F7F4FD2
S1130DD080E00E94FA048B8183FD10E08FB7F894C1
S1130DE0112319F023E030E002C025E030E0309315
S1130DF02801209327018FBFC09A112331F082E08C
S1130E000E9446060E94B0040CC00E94C702DC0186
S1130E10CB0120E431E040E050E0BC01CD010E9470
S1130E20920423960FB6F894DEBF0FBECDBFDF91B8
S1130E30CF911F9108952F923F924F925F926F929C
S1130E407F928F929F92AF92BF92CF92DF92EF9256
S1130E50FF920F931F93CF93DF93CDB7DEB72E97F7
S1130E600FB6F894DEBF0FBECDBF6E837F83888735
S1130E7099877FEF272E7FEF372E7FEF472E7FEF67
S1130E80572E1A861B861C8664E3662E61E0762E36
S1130E90F301608561FFE9C0E080F1800281138184
S1130EA08E819F81A885B9858E199F09A00BB10BEE
S1130EB0248135814681578149015A01881A990A4A
S1130EC0AA0ABB0AF1E0FD87B7FDC2C082179307E7
S1130ED0A407B50708F4BCC060FF05C06D7FF3012B
S1130EE060871D860DC0E20EF31E041F151FF3015B
S1130EF0E082F18202831383820E931EA41EB51E28
S1130F008B85E82EFF24E114F10409F09EC08FB70D
S1130F10F8949927C0902D01CC2011F08FBF95C073
S1130F208FBF80B3992756E0969587955A95E1F738
S1130F30F82FF170FE878091CF0590913E018917BB
S1130F4009F47DC0F91709F07AC084E090E0909329
S1130F502F0180932E018E010F5F1F4F80910E0190
S1130F6090910F018983892F9927F80181838091BA
S1130F70C4069091C5068B83892F99278C838FB7DC
S1130F80F894992721E0D22ED0922D018FBF87E0CB
S1130F900E948A01B7018DE10E94010524E0A801A5
S1130FA06C2D88E691E00E942E05C09AC0988FB7F8
S1130FB0F894E82EFF248D2D0E94E70401E010E050
S1130FC01093280100932701C0922601C092B9060C
S1130FD0EFBE8FB7F894E82EFF240E94910210937D
S1130FE053010093520189B78F7B89BF80E488BF86
S1130FF08AB780628ABF8AB78F7E8ABF89B78064C6
S113100089BFEFBE8FB7F894082F112780912E0166
S113101090912F01049731F4BE016B5F7F4F83E001
S11310200E94FA040FBF8FB7F894082F1127C09AB3
S113103080E00E9446060FBF82E00E948A01FE857E
S1131040F093CF0586E00E948A012D85222369F062
S1131050F301808581FF09C082149304A404B504BC
S113106010F414012501F1E0FA872B853C852F5FEC
S11310703F4F2B873C8749E050E0640E751E1216E3
S113108013060CF005CF5A85552391F10E949B025B
S11310907B018C012E813F8148855985621B730B2E
S11310A0840B950B621573058405950520F089E082
S11310B00E948A011DC0261A370A480A590AE0927A
S11310C0AF06F092B0060093B1061093B2062092D8
S11310D0AB063092AC064092AD065092AE0621E0CB
S11310E020933D01A2019101C801B7010E94BE03F2
S11310F02E960FB6F894DEBF0FBECDBFDF91CF9111
S11311001F910F91FF90EF90DF90CF90BF90AF9021
S11311109F908F907F906F905F904F903F902F9013
S113112008956F927F928F929F92AF92BF92CF92C7
S1131130DF92EF92FF920F931F93CF93DF93CDB77C
S1131140DEB721970FB6F894DEBF0FBECDBF8FB7C1
S1131150F894A090CD05B090CE05609046017090B3
S1131160470100914D0110914E01A801465F5F4F68
S113117020915B0630915C062417350708F09A012C
S11311808FBF49010894810891080815190530F5A5
S11311906801C60CD71C7801EA0CFB1CA114B1042D
S11311A031F0BE016F5F7F4FF701808104C0BE0143
S11311B06F5F7F4F80E00E94FA046114710419F09C
S11311C08981F60180830F5F1F4F0894E11CF11C95
S11311D00894C11CD11C0815190500F381E00E9474
S11311E070058FB7F894982FA114B10431F0A00EB4
S11311F0B11EF50180818FB901C01FB810934E0153
S113120000934D019FBF80E090E021960FB6F894C3
S1131210DEBF0FBECDBFDF91CF911F910F91FF9025
S1131220EF90DF90CF90BF90AF909F908F907F9082
S11312306F9008959C018FB7F89499273093CE0549
S11312402093CD05709347016093460150935C064B
S113125040935B0610924E0110924D018FBF8FB1E7
S11312600E949108992708950F931F93CF93DF93BA
S1131270CDB7DEB721970FB6F894DEBF0FBECDBF52
S1131280C09800913201109133018FE790E0909360
S11312908D0680938C06BE016F5F7F4F80918C0614
S11312A00E94FA0441E050E0B80180E090E00E941E
S11312B01A0921960FB6F894DEBF0FBECDBFDF9199
S11312C0CF911F910F91089582E090E09093530184
S11312D08093520183E00E948D05882319F40E94B3
S11312E03409089583E00E9414060895CF938FB7BC
S11312F0F894282F3327C22F8091520190915301E3
S1131300892B11F42FBF26C02091DD06222341F042
S113131080E090E0B79B02C081E090E0892B49F423
S113132081B19927E6E096958795EA95E1F780FDE6
S113133008C0222319F021502093DD060E9464097D
S113134008C081E090E09093530180935201109281
S1131350DD06CFBFCF910895EF92FF921F93CF93F5
S1131360DF93CDB7DEB721970FB6F894DEBF0FBE7B
S1131370CDBFE0909B03F0909C03F70187A19927D0
S1131380182F882309F41FE1C0988091B9068117AA
S113139041F0812F9927806E9068BC0185E10E94FD
S11313A001051093B906F701108111508EE390E006
S11313B090938D0680938C06BE016F5F7F4F809162
S11313C08C060E94FA04812F9927AC0160E070E03A
S11313D0C7010E941A0921960FB6F894DEBF0FBE0A
S11313E0CDBFDF91CF911F91FF90EF900895982F7B
S11313F080911901882399F5992389F531E0309377
S11314001901809106018093180120912401822FF3
S11314108323809350018091000190910101909366
S113142017018093160180912301809315013227BF
S113143031702E7F232B822F8170E82FFF27EE0F30
S1131440FF1FEE5FFE4F8081918190930101809395
S11314500001277E2093240181E10E948A010895DE
S1131460982F8D57823070F480911401816080939D
S1131470140180E289278093CC058DE70E94AF0197
S113148099270895892F0E94AF0199270895262F3F
S1131490E6EBF0E02927220FF11DE20FF11DC895BC
S11314A0982F802D3196C895902508951F93CF933A
S11314B0182FC62F8091E30599278130910509F1F2
S11314C0823091051CF4009749F041C182309105A6
S11314D009F454C0039709F464C039C1112309F411
S11314E05DC1109242011092410110928B0610923C
S11314F090061092D3059093400180933F0181E0C0
S11315004DC0112309F04AC180913F0190914001DF
S11315100E94470A9093400180933F0182E08093A8
S1131520E305C0939006C43409F011C1C43409F032
S11315300EC1212F8091240180FF03C0982F96951E
S113154003C0982F96959695917099F480FF02C0E8
S1131550846001C082608093240180912401877E8D
S1131560886080932401109223018FEF80930601F9
S113157001C025E0222309F411C1E9C0112309F0B7
S11315806AC06093D30580913F01909140010E940D
S1131590470A9093400180933F0183E08093E305E1
S11315A0FDC080918B068F3F09F4C8C0112309F454
S11315B05CC0823008F44FC090914101992319F026
S11315C0E92FE15001C0E2E09E2FFF27EF5BFE4FC1
S11315D08281282F3327322F2227992319F0E92FCC
S11315E0E15001C0E2E0FF27EF5BFE4F82819927C3
S11315F0282B392B80913F019091400128173907FE
S113160001F580E00E94F7093091D3058091BB0673
S11316102091BC06982F9F5F963008F090E09217B7
S113162009F495C0E82FFF27E554F94F32838F5F03
S11316308093BB06863010F01092BB060E94DC013A
S113164086C080915E0190915F01019690935F0145
S113165080935E017CC08091620190916301019648
S1131660909363018093620172C0823008F452C087
S113167080914201E82FFF27EF5BFE4F8281482FC4
S11316805527342F20912401822F8695869586959F
S1131690837099278130910519F0029781F01FC05A
S11316A0822F877E806180932401442311F486E095
S11316B001C080E0809323013093060110C0809123
S11316C023018E3260F4E0910001F0910101E80FF2
S11316D0F11D4083809123018F5F809323018091CA
S11316E04201E82FFF27EF5BFE4F92818F5F8093CB
S11316F04201833010F010924201892F9927682FFC
S113170080913F01909140010E94470A90934001CB
S113171080933F0180914101E82FFF27EF5BFE4F4B
S1131720C2838F5F80934101833010F01092410196
S113173080918B068F5F80938B0630C0809164010B
S113174090916501019690936501809364011092D4
S11317504201109241011092E30510928B061092FF
S113176090061092D3051092400110923F0180918F
S113177014018D7F80931401C1E08C2F0E94F7091E
S113178080912501882331F084E08093E3050E9451
S1131790B90104C0112311F0C093E305CF911F9147
S11317A00895CF92DF92EF92FF920F931F93CF93FE
S11317B0DF93CDB7DEB725970FB6F894DEBF0FBE23
S11317C0CDBF9927AA27BB27FC01429708F0DEC4A6
S11317D0EA5BFF4FEE0FFF1F0590F491E02D099493
S11317E08FB7F894282F3327922F80919A03E09192
S11317F0E1058E1739F480915A06882319F48093F1
S1131800DA06AFC19FBFFF27EE0FFF1FEF56F94F58
S1131810E080F180F70180818C50082F112700931C
S1131820AA06C7010E94C302D7011696FD01918141
S1131830292F3327322F2227F7019681492F552745
S1131840242B352BFD012183232F3327F7012683F6
S11318508287008782E28187C0901F01D090200197
S1131860C114D10419F085E090E040C082E090E01A
S11318709093200180931F0110921A0110921B0172
S11318808FB7F894482F552710921C01F09222012B
S1131890E092210186E090E080931D010B5F080F28
S11318A000931E014FBF90E08FB7F894282F332781
S11318B08091DF05882331F481E08093DF059093E4
S11318C0E005982F2FBF992321F00E94DC01C60167
S11318D002C085E090E0882319F480E090E006C01F
S11318E01092200110921F0181E090E0892B09F0F1
S11318F0CEC38FB7F894282F33278BB392E0B4C0AC
S11319008FB7F894282F3327922F8091E205E09126
S11319104C018E1739F48091D905882319F48093EA
S113192051011FC19FBFFF27EE0FFF1FEA51FA4F5E
S1131930C080D180A6014A5F5F4F18E0E12EF12CF0
S1131940EC0CFD1CF601108586819927982F8827B9
S1131950FA0121813327822B932BF6018683892F69
S11319609927FA01818382E290E0F601848360E0A2
S113197070E06583145F8FB7F894282F3327809124
S11319803101833021F02FBF81E090E065C085E014
S113199080933101D092D906C092D8068091A906CD
S11319A08F5F8093A906F60183832FBFD6011D9311
S11319B081E498E8818388E890E0FD018183FA015D
S11319C081819927982F8827F60126813327822B36
S11319D0932B8F5F9F4F51F0F6018181992780628D
S11319E098688183892F9927FD018183809107015C
S11319F090910801F6018087892F9927F701818347
S1131A00F60163A760A761A715A664A74091D8064D
S1131A105091D9068FB7F894282F33278091270146
S1131A2090912801019711F02FBF14C082E090E03B
S1131A30909328018093270181E08093CA055093F5
S1131A409C0340939B032FBF0E943706882311F405
S1131A500E94AC0980E090E0892B11F58FB7F894CF
S1131A60282F33278BB394E089278BBB7AC083E07C
S1131A70809331011092D90589C381E080933101AB
S1131A8085C38FB7F8949927309130018FBF83E0D5
S1131A90809331014091D8065091D906332319F02F
S1131AA00E9480011FC08FB7F894682F20914C01C9
S1131AB0E22FFF27EE0FFF1FEA51FA4F8081918139
S1131AC04817590771F4822F8F5F80934C018C3033
S1131AD010F030934C018091D905882311F0309394
S1131AE0D9056FBF81E0F6C28FB7F8949927109299
S1131AF04F014BC38FB7F894082F112780912D0104
S1131B00882301F50E949B02DC01CB018093340100
S1131B1090933501A0933601B093370181E090E0B2
S1131B20A0E0B0E08093380190933901A0933A018A
S1131B30B0933B0180913C01836080933C0189E038
S1131B400E948A010FBF22C38FB7F894282F33272E
S1131B5080912D01882329F080913C018D7F809311
S1131B603C012FBF13C340913D01442379F58FB746
S1131B70F894282F3327E090C605F090C70500910C
S1131B80C8051091C9058091920390919303A09187
S1131B909403B0919503E80EF91E0A1F1B1F2FBF73
S1131BA08091AB069091AC06A091AD06B091AE06C3
S1131BB0E092AF06F092B0060093B1061093B2061D
S1131BC09C01AD01C801B7010E94BE038091AF061C
S1131BD09091B006A091B106B091B2062091AB06E7
S1131BE03091AC064091AD065091AE06820F931F22
S1131BF0A41FB51F07C087B78D7F87BF0E949B02B4
S1131C00DC01CB01BC01CD010E941B07BFC28FB711
S1131C10F894282F332790910B0190930C0182E0C4
S1131C2080932A012FBF992309F0B0C28FB7F8948B
S1131C30992720910D018FBF33272130310509F4F5
S1131C4056C0223031051CF4232B51F09FC22230A0
S1131C50310509F47EC02330310509F492C096C2DF
S1131C60C0988FB7F894E82EFF2480912E019091AC
S1131C702F010297D1F583E090E090932F01809398
S1131C802E0168E170E08DE10E94010511E01093DE
S1131C903E0110922D0180B3992766E096958795B1
S1131CA06A95E1F781238093CF0586E00E948A013B
S1131CB0BE016F5F7F4F812F0E94FA046FE772E0CD
S1131CC08CE10E9401059091100185E0989FC0016C
S1131CD01124825D9E4F9064BC0188E10E9401053D
S1131CE062EF7AE281E10E940105EFBE4FC28FB735
S1131CF0F894282F3327409110018E010E5F1F4F57
S1131D0080910E0190910F018A83892F99278B83EB
S1131D108091C4069091C506F8018283892F992782
S1131D2083832FBFC09885E0F82E4F9DC0011124F6
S1131D30825D9E4F9064BC0188E10E94010524E00D
S1131D40A80160E088E691E00E942E05C09A8F2DDC
S1131D50C1C18FB7F8949927209127018FBF3327EA
S1131D602230310521F02430310521F006C00E94D3
S1131D70AC090CC20E94C30609C282E00E94460656
S1131D8005C20E94340902C28FB7F8949927FDC195
S1131D90A0913201B09133018C919D01280F311D26
S1131DA0F9018081881F8827881FFD0182A7F90116
S1131DB082919F012F5F3F4FFD0180A7F901808130
S1131DC08F77FD0181A7A0913201B0913301FD010C
S1131DD087819927382F222786819927282B392B09
S1131DE080910701909108012817390719F02F5F96
S1131DF03F4F91F58D018FB7F894F82E80915A06D4
S1131E00882329F580919A039927FC01E80FF91F8B
S1131E10EF56F94F00811181A083B18301966CE0E4
S1131E2070E00E94501A80939A03982F8091E105E4
S1131E30981719F481E080935A068091DA06882372
S1131E4041F40E948A0181E08093DA0602C00E9474
S1131E508001FFBEF80101C0FD01F0933301E0935E
S1131E6032010E94760992C1A0E0BA2F1A2F8FB7CF
S1131E70F894282FA0939D033A2F8091B7068823C6
S1131E8009F431E0412F883009F441E0912F893081
S1131E9009F491E0442311F4992359F01093B706FF
S1131EA08091B806E82FFF27EE0FFF1FE352FA4F89
S1131EB010832FBF442311F4992391F1992371F0D6
S1131EC08FB7F894282F3327809160019091610196
S1131ED0019690936101809360012FBF8091DA0590
S1131EE08F5F8093DA058091BA06833499F48FB7B3
S1131EF0F894282F8091BB069091BC06891741F075
S1131F00892F8F5F8093BC06863010F01092BC0638
S1131F102FBF09C0A0E0442309F4A1E0B1E003C04D
S1131F20332309F452C08FB7F894992730912501CF
S1131F308FBF332349F08FB7F894282F33278AE0D3
S1131F408093B7062FBF41C08FB7F894992760914B
S1131F50DD052091DF058FBF8FB7F8949927709125
S1131F60BB06E091BC067E1709F431E08FBF332332
S1131F7011F5662301F58FB7F894482F552782E0B1
S1131F808093DD05262F8FB7F8949927362F7E1777
S1131F9009F431E08FBF332321F4FF27E554F94FCF
S1131FA022812093DE054FBF83E48093BA066093B9
S1131FB0B80611E00AC02150223038F485E4809339
S1131FC0BA0681E08093B806182FBB2349F08FB777
S1131FD0F8949927A0931C018FBF80E10E948A0185
S1131FE08091B7068A3019F40E94B901CFC0112339
S1131FF009F4CCC08FB7F894282F33271092D10559
S11320001092D0051092D20581E08093B7062FBFBD
S1132010809114018E7F809314018EE70E94AF019A
S1132020882309F4B3C08FB7F894282F332789E0A5
S11320308093B7062FBF0E94DC01A8C08AB18069D3
S11320408AB98AB188648AB910925A069FC08AB143
S11320508F768AB98AB1877B8AB998C01092200199
S113206010921F018FB7F894992730911C018FBFEC
S113207080911B01811133E080911A01409121016B
S113208050912201882309F081C0332319F00E9462
S113209080011FC08FB7F894682F2091E105E22FCB
S11320A0FF27EE0FFF1FEF56F94F808191814817EC
S11320B0590771F4822F8F5F8093E1058C3010F003
S11320C03093E10580915A06882311F030935A0623
S11320D06FBF80E00E948A0159C08FB7F894992796
S11320E0209118014091160150911701E090500180
S11320F08FBF2223A1F58A018FB7F894F82E90910F
S1132100D905992339F58091E205E82FFF27EE0FD1
S1132110FF1FEA51FA4F00811181408351838F5F81
S11321208093E2058C3010F09093E2059091E205E3
S113213080914C01981719F481E08093D90580911E
S11321405101882349F481E00E948A0181E080934F
S1132150510102C00E948001FFBE980101C09A0192
S11321608FB7F894EE2DFF27EE0FFF1FEE5FFE4FA3
S11321702083318390912401EE2011F09B7F01C0D4
S11321809D7F90932401109219018FBF25960FB65D
S1132190F894DEBF0FBECDBFDF91CF911F910F9199
S11321A0FF90EF90DF90CF9008958091C3068F3F0A
S11321B0D1F09091C3068091C306E82FFF27EA531C
S11321C0F94F80818093C3068091C3068F3F11F439
S11321D08093DB06892F9927FC01EA53F94F2FEFEF
S11321E020839C0102C02FEF30E02F3F19F480E0E0
S11321F090E00895822F0E94D10B81E090E0089531
S1132200CFEFD0E1DEBFCDBF8FB7F894182F42E1F6
S113221050E06FEF70E086EC96E00E94491A8FEF71
S11322208093C3068093DB0681E08EBD88E080BF87
S113223083E083BF2CB53DB54AE78CB59DB58217C5
S1132240930708F441509C014423B9F792B782B72D
S11322508917E9F32CB53DB592B782B78917E9F32D
S11322608CB59DB5821B930B409675E0969587952A
S11322707A95E1F79093DC058093DB0513BE83B771
S11322808EBD8EB580BF12BE1DBC1CBC8FEF86BF39
S113229086B780937C0080B7282F3327277030704F
S11322A021153105C1F7D29AD19AD09ADA9AD99ADE
S11322B0D89A25BB8FEF84BBD498DC9880B788600C
S11322C080BF3DBD2CBD87B7846087BF8EB5887F36
S11322D084608EBD80E285BF0E94D510C82FDD27A3
S11322E0CC23D1F7C093DD05C093DF05C093B706B7
S11322F0C093D205C093BA06C093DA051092D105F3
S11323001092D005C0939D03C093B806C0934201B8
S1132310C0934101C093E305C0938B06C09390061C
S1132320C093D3051092400110923F01C093BC06A4
S1132330C093BB0682E1E4E5F1E011928A95E9F7E6
S1132340C09357018FEF90E0909359018093580107
S113235081E0809354018091DB059091DC05AA27EC
S1132360BB276CE0880F991FAA1FBB1F6A95D1F782
S1132370BC01CD0120E031EE40E050E00E94631A40
S1132380DA01C901019789B9892F992780939000AF
S113239082E08BB986E080939500CAB980911101DF
S11323A0909112010196AA27BB2780938E039093E4
S11323B08F03A0939003B093910300B602FCFDCF6A
S11323C012BE87B7816087BF83B7887F836000B6FA
S11323D000FCFDCF83BF80913101882319F481E093
S11323E080933101B89AD69AD59A80910701909139
S11323F008019093C5068093C4068E98B89A8C9869
S11324008DE596E090933301809332010E94D510BC
S11324108823E1F71FBF789486E691E02BE0E1E999
S1132420F6E08193919321508E9627FFFACF109274
S1132430E10510929A031092DA0681E080935A061D
S11324408EE993E02BE0E6EEF5E081939193215041
S11324508E9627FFFACF10924C011092E20510924B
S1132460510181E08093D90580913101813049F592
S113247082E0809331010E94FF01DC01CB01809353
S1132480A9068FB7F894282F332780912E019091B5
S11324902F01892B11F02FBF14C081E090E090939D
S11324A02F0180932E012FBFDD9A0E94C702DC0109
S11324B0CB0124E130E040E050E0BC01CD010E94BA
S11324C092048EE00E948A018FB7F894482F4CC082
S11324D087B79927887B892B41F480917D00282F29
S11324E033272B7F2115310519F020E030E02CC073
S11324F06F992AC08AB1807C39F580919A00807CDA
S113250019F5379B03C021E030E01EC087B7992737
S113251083709070892BB1F083B783BF80B79927FC
S113252087709070892BD1F781B792B7891B80315E
S113253018F082B7813F18F022E030E005C023E0B4
S113254030E002C025E030E0E5E02E1708F4E22F89
S113255085B7837EFF27E055FF4F9491892B8062D6
S113256085BF78948895F8948091C3068F3FC9F00D
S11325709091C3068091C306E82FFF27EA53F94FD1
S113258080818093C3068091C3068F3F11F48093AA
S1132590DB06892F9927FC01EA53F94F2FEF20839B
S11325A002C08FEF90E08F3F09F492CF4FBF0E949B
S11325B0D10B8ACF83B783BF00B600FCFDCF08954B
S11325C01F920F920FB60F9211242F933F934F93A4
S11325D05F936F937F938F939F93AF93BF93CF93A7
S11325E0EF93FF930E94DA12789487B78D7F87BFA9
S11325F08FB7F894C82F8091920390919303A09180
S11326009403B09195030097A105B10521F488E0E6
S11326100E948A0102C00E94E602CFBFFF91EF919F
S1132620CF91BF91AF919F918F917F916F915F9166
S11326304F913F912F910F900FBE0F901F901895BF
S11326401F920F920FB60F9211242F933F934F9323
S11326505F936F937F938F939F93AF93BF93EF9306
S1132660FF930E94DA1281E08093E5058091D505FD
S11326709091D605A091D705B091D8050196A11DDA
S1132680B11D8093D5059093D605A093D705B0933B
S1132690D8058091CB05882339F081508093CB05F0
S11326A0882311F40E94E6021092E505FF91EF9150
S11326B0BF91AF919F918F917F916F915F914F9156
S11326C03F912F910F900FBE0F901F901895789403
S11326D01F920F920FB60F9211241F932F933F93C3
S11326E04F935F936F937F938F939F93AF93BF9316
S11326F0EF93FF93CF93DF93CDB7DEB72197F89491
S1132700DEBF7894CDBF87B78F7E87BF8FB7F8942D
S1132710182F8091B3069091B406A091B506B0919C
S1132720B6060097A105B10509F06DC08091270197
S1132730909128018430910561F18530910518F458
S1132740039739F04EC08530910599F1079741F10F
S113275048C080B39927689415F896958795169480
S1132760E1F780FF13C084E090E090932801809308
S113277027010E94C702DC01CB0127E030E040E0E2
S113278050E0BC01CD010E9492042BC00E94B00411
S113279028C00E943706882321F50E94C30621C061
S11327A081E090E0909328018093270110923001FA
S11327B015C0BE016F5F7F4F89E00E94FA0487B79E
S11327C08F7D87BF81E00E94E70481E090E09093D1
S11327D028018093270187E08093300184E00E94E0
S11327E08A0180912E0190912F01019771F482E06A
S11327F090E090932F0180932E01DE98DE9A80E082
S11328000E94140602C00E94DC031FBF2196F894A4
S1132810DEBFCDBFDF91CF91FF91EF91BF91AF911B
S11328209F918F917F916F915F914F913F912F91E4
S11328301F910F900FBE0F901F90189578941F92C0
S11328400F920FB60F9211240F900FBE0F901F908E
S1132850189578941F920F920FB60F9211240F902F
S11328600FBE0F901F90189578941F920F920FB679
S11328700F9211241F932F933F934F935F936F9362
S11328807F938F939F93AF93BF93CF93DF93EF93F4
S1132890FF93CCB5DDB580E286BF8FB7F894182FCF
S11328A080912701909128018530910519F00697B0
S11328B039F157C080E00E94E70482E00E94460696
S11328C087B78F7E87BF86E090E09093280180933E
S11328D02701E0919B03F0919C03818199278770E4
S11328E09070019721F4C5A78D2F992784A780B3F1
S11328F09927B4E096958795BA95E1F780FD77C05E
S113290081E00E94E704E0919B03F0919C038181A4
S113291085FF13C087E090E09093280180932701FE
S11329200E94C702DC01CB0120E830E040E050E027
S1132930BC01CD010E9492040BC081E090E0909311
S11329402801809327011092300184E00E948A01BB
S113295080B39927A4E096958795AA95E1F780FF1F
S113296046C080912601882351F50E94E7044091D6
S1132970E4054830A0F48091D405840F912D911D75
S11329809C01887F9370281BE22FFF27EE0FFF1F07
S1132990E252F94FC083D1834F5F4093E40581E055
S11329A080932601D0938F06C0938E0680B3992717
S11329B0F4E096958795FA95E1F780FD18C080912B
S11329C026018823A1F081E00E94E70410922601E9
S11329D080918E0690918F06C81BD90B2A9738F4E4
S11329E08091E405882319F081508093E4051FBF8A
S11329F0FF91EF91DF91CF91BF91AF919F918F9113
S1132A007F916F915F914F913F912F911F910F9003
S1132A100FBE0F901F90189578941F920F920FB6C7
S1132A200F9211242F933F938F939F938FB7F89412
S1132A30282F33278091490190914A010196909360
S1132A404A01809349012FBF9F918F913F912F910C
S1132A500F900FBE0F901F9018951F920F920FB6F4
S1132A600F9211240F900FBE0F901F9018951F9274
S1132A700F920FB60F9211240F900FBE0F901F905C
S1132A8018951F920F920FB60F9211240F900FBE3C
S1132A900F901F9018951F920F920FB60F9211244A
S1132AA00F900FBE0F901F9018951F920F920FB6A4
S1132AB00F9211240F900FBE0F901F9018951F9224
S1132AC00F920FB60F9211240F900FBE0F901F900C
S1132AD018951F920F920FB60F9211242F933F93C4
S1132AE04F935F936F937F938F939F93AF93BF9312
S1132AF0EF93FF938091520190915301019719F440
S1132B000E94640905C08091DD068F5F8093DD0615
S1132B10FF91EF91BF91AF919F918F917F916F91B1
S1132B205F914F913F912F910F900FBE0F901F9087
S1132B3018951F920F920FB60F9211240F900FBE8B
S1132B400F901F9018951F920F920FB60F92112499
S1132B50CF92DF92EF92FF920F931F932F933F93A5
S1132B604F935F936F937F938F939F93AF93BF9391
S1132B70EF93FF93CF93DF93CDB7DEB72297DEBFFA
S1132B80CDBF8FB1282F3327E0914601F091470143
S1132B90309739F080914D0190914E01E80FF91F63
S1132BA0208380914D0190914E01019690934E01A6
S1132BB080934D0180E00E94700520914D01309179
S1132BC04E0180915B0690915C062817390718F432
S1132BD00E9491084BC1C0904601D09047011092C9
S1132BE04701109246011092CE051092CD05109225
S1132BF05C0610925B0610924E0110924D018FB14B
S1132C0080918C0690918D0620918C0686FFE9C0F8
S1132C102F7B822F99278E33910509F427C1CF97F3
S1132C2009F024C10091320110913301F801E080D0
S1132C3080915201909153018230910521F00397C4
S1132C4009F44BC0C9C083E090E090935301809392
S1132C5052014E2D55279A012F5F3F4F6091480135
S1132C60862F992782179307ACF40E949102C09A89
S1132C70C098BE016F5F7F4F88E00E94FA04BE01D6
S1132C806E5F7F4F88E00E94FA04C09A83E00E943E
S1132C9046069FC080E090E0B79B02C081E090E0D0
S1132CA0892B69F481B1992776E0969587957A9571
S1132CB0E1F780FD04C06E19615060934801F8E2A9
S1132CC0FE1520F0B8016F5F7F4F02C060E070E036
S1132CD080E090E00E941A09C9C0C09A83E00E9473
S1132CE046068091E405882319F18AE08E1538F5AB
S1132CF08091D405E82FFF27EE0FFF1FE252F94F12
S1132D0080819181F80185A7892F992784A78091D3
S1132D10D405992701969C01287F3170821B930B5F
S1132D208093D4058091E40581508093E40507C025
S1132D308FEF9FEFF80185A78FEF90E084A7F8014C
S1132D40EE0DF11D808187FF44C0CD2809F441C0F8
S1132D50F801618167704091320150913301623012
S1132D6091F5A0919B03B0919C03FA01208180917D
S1132D70270190912801079761F5FD019381FA01DC
S1132D808381891731F587B78F7E87BF81E0FD0185
S1132D9083A7420F511DFA0182919F012F5F3F4F7C
S1132DA0FD0180A7F90180818F77FD0181A781E072
S1132DB090E090932801809327011092300184E0E1
S1132DC00E948A0106C0613021F48CE00E948A01CD
S1132DD04DC00E9476094AC0C09A83E00E9446060C
S1132DE045C02E3309F042C0C09A809127019091CA
S1132DF02801089739F481E090E0909328018093AA
S1132E00270134C08091CA05882349F484E090E006
S1132E1090932801809327010E94C30627C082E073
S1132E200E94460683E090E0909328018093270156
S1132E300E94FF01DC01CB018F71907001969C010F
S1132E4043E0220F331F4A95E1F7280F391F280F5B
S1132E50391F7901002711270E94C702DC01CB0129
S1132E60A8019701BC01CD010E9492042296F89416
S1132E70DEBFCDBFDF91CF91FF91EF91BF91AF91B5
S1132E809F918F917F916F915F914F913F912F917E
S1132E901F910F91FF90EF90DF90CF900F900FBE96
S1132EA00F901F9018951F920F920FB60F92112436
S1132EB02F933F934F935F936F937F938F939F933E
S1132EC0AF93BF93EF93FF935F9B18C06CB16E37C2
S1132ED019F460E081E010C0809114016D3721F491
S1132EE08260809314010AC081FF05C08D7F8093A6
S1132EF0140180E2682780E00E94560AFF91EF9156
S1132F00BF91AF919F918F917F916F915F914F91FD
S1132F103F912F910F900FBE0F901F9018951F9205
S1132F200F920FB60F9211248F9380919B0087FF0D
S1132F3002C080919C008F910F900FBE0F901F9044
S1132F40189578941F920F920FB60F9211241F9325
S1132F502F933F934F935F936F937F938F939F939D
S1132F60AF93BF93CF93EF93FF932091140120FF6E
S1132F7008C02E7F209314018091CC050E94AF01DC
S1132F80BBC08091B70699278430910509F492C09B
S1132F90853091054CF48230910509F18330910517
S1132FA09CF5019789F0A3C08630910509F490C07F
S1132FB0863091050CF485C08730910509F493C0DF
S1132FC0089709F497C093C08091BA060E94300A0A
S1132FD0C82F83E08093B7066091BA060AC0809137
S1132FE0DA050E94300AC82F83E08093B706609107
S1132FF0DA058091D0059091D1050E94470A9093FB
S1133000D1058093D00571C08FB7F894182F8091A3
S1133010B806E82FFF27EE0FFF1FE252FA4F808118
S11330200E94300AC82F8091B806E82FFF27EE0FC0
S1133030FF1FE252FA4F60818091D0059091D10533
S11330400E94470A9093D1058093D0058091D205C0
S11330508F5F8093D2058091B806813031F58091DD
S11330601D01E0912101F0912201E80FF11DE081A1
S1133070982F9F5F90931D0180911E01891730F452
S113308082E08093DF0580E090E002C08E2F9927D4
S1133090E82FFF278091DF05823039F08091D20537
S11330A08F3F19F0E093E00503C084E08093B706F6
S11330B01FBF1BC08091D0050E94300AC82F85E035
S11330C00FC08091D1050E94300AC82F86E008C045
S11330D02E7F209314018EE70E94AF01C82F87E052
S11330E08093B70602C088E003C0CC2329F089E0AE
S11330F08093B7060E94DC01FF91EF91CF91BF91BD
S1133100AF919F918F917F916F915F914F913F917B
S11331102F911F910F900FBE0F901F9018957894C8
S11331201F920F920FB60F9211240F900FBE0F90A3
S11331301F901895A0E3B0E0E0EAF8E10C94B81A07
S1133140222E332E442E552E662E772E882E992E1F
S11331502A2D3B2DA8E0FE013196AA2E1192AA94A5
S1133160E9F729823A824B825C826D827E828F8269
S11331709886FE013996BA2E1192BA94E9F72987F6
S11331803A87CB86DC86ED86FE860F87188BFE0198
S113319071961192AA95E9F7C980DA80EB80FC80D8
S11331A0C9A6DAA6EBA6FCA6870176018FEF9FEFEE
S11331B0A0E0B0E0E822F9220A231B23A9A4BAA4C0
S11331C0CBA4DCA416014424552489859A85AB85B7
S11331D0BC858DA79EA7AFA7B8AB5C016D018FEF2F
S11331E09FEFA0E0B0E0A822B922CA22DB228DA57D
S11331F09EA5AFA5B8A93D0188249924C801B701AB
S1133200A60195010E94851A69A37AA38BA39CA3A6
S1133210C801B701A40193010E94851A6DA37EA37E
S11332208FA398A7C201B101A60195010E94851A36
S11332307B018C01C201B101A40193010E94851A92
S11332409B01AC01A9A0BAA0CBA0DCA0C601AA270F
S1133250BB27ADA0BEA0CFA0D8A4A80EB91ECA1E7D
S1133260DB1EAE0CBF1CC01ED11EADA2BEA2CFA2DF
S1133270D8A6AE14BF04C006D10620F420503040B6
S11332804F4F5F4FCDA0DEA0EFA0F8A4C701AA273F
S1133290BB27820F931FA41FB51F8D8F9E8FAF8FE7
S11332A0B8A3A6013327222789A19AA1ABA1BCA167
S11332B0A070B070280F391F4A1F5B1F298F3A8FE7
S11332C04B8F5C8FA98CBA8CCB8CDC8CED8CFE8CF8
S11332D00F8D18A1ED8AFE8A0F8B188F2D853E85E0
S11332E04F85588969A57AA58BA59CA50E94851A46
S11332F03B014C018D819E81AF81B885BC01CD011C
S11333002DA53EA54FA558A90E94851ADC01CB0125
S1133310680E791E8A1E9B1E8D899E89AF89B88D81
S1133320860D971DA81DB91D8D8B9E8BAF8BB88FF5
S11333306D897E898F89988D2A2D3B2D4C2D5D2D8D
S1133340E2E1E0960C94D41A8F929F92AF92BF92CE
S1133350CF92DF92EF92FF920F93CF93DF93CDB78B
S1133360DEB768970FB6F894DEBF0FBECDBFE82E68
S1133370002349F4298B3A8B4B8B5C8B6D8B7E8BB2
S11333808F8B988F6CC088E0FE01319611928A95DC
S1133390E9F729833A834B835C836D837E83EF82D1
S11333A0988740E2401B14160CF041C08D819E8129
S11333B0AF81B8856C017D0104C0CC0CDD1CEE1C12
S11333C0FF1C4A95D2F7202F332727FD3095022E74
S11333D004C0B695A795979587950A94D2F78D87DB
S11333E09E87AF87B88B89819A81AB81BC8104C0E9
S11333F0B695A795979587952A95D2F78C299D29F7
S1133400AE29BF2989879A87AB87BC8729853A85E6
S11334104B855C856D857E858F859889298B3A8B54
S11334204B8B5C8B6D8B7E8B8F8B988F18C01D861E
S11334301E861F86188A842F992787FD9095222738
S11334403327281B390B8D819E81AF81B88504C039
S1133450B695A795979587952A95D2F7D3CF2989BD
S11334603A894B895C896D897E898F89988D6896A4
S11334700FB6F894DEBF0FBECDBFDF91CF910F9191
S1133480FF90EF90DF90CF90BF90AF909F908F9080
S11334900895DC0101C06D9341505040E0F7089558
S11334A097FB092E07260AD077FD04D04DD006D00D
S11334B000201AF4709561957F4F0895F6F7909562
S11334C081959F4F0895A1E21A2EAA1BBB1BFD01F3
S11334D00DC0AA1FBB1FEE1FFF1FA217B307E407EF
S11334E0F50720F0A21BB30BE40BF50B661F771F47
S11334F0881F991F1A9469F7609570958095909527
S11335009B01AC01BD01CF010895629FD001739F5F
S1133510F001829FE00DF11D649FE00DF11D929F6B
S1133520F00D839FF00D749FF00D659FF00D9927AA
S1133530729FB00DE11DF91F639FB00DE11DF91FCE
S1133540BD01CF0111240895AA1BBB1B51E107C083
S1133550AA1FBB1FA617B70710F0A61BB70B881F1F
S1133560991F5A95A9F780959095BC01CD010895AE
S11335702F923F924F925F926F927F928F929F927F
S1133580AF92BF92CF92DF92EF92FF920F931F936D
S1133590CF93DF93CDB7DEB7CA1BDB0B0FB6F8941E
S11335A0DEBF0FBECDBF09942A88398848885F845E
S11335B06E847D848C849B84AA84B984C884DF80CF
S11335C0EE80FD800C811B81AA81B981CE0FD11DB3
S11135D00FB6F894DEBF0FBECDBFED01089517
S11335DEFE05FE052C06FF0100FFFFFFFFFF220084
S10735EE1A010000BA
S9030000FC
